:1000000058C064C271C070C06FC06EC06DC06CC09B
:100010006BC06AC069C068C067C066C065C064C0A4
:1000200063C062C061C00403090422037700770043
:1000300077002E0072006500630075007200730087
:1000400069006F006E002E006A00700010035500FA
:10005000530042002D00500049004F0012010101E1
:1000600002000008C016E1050001010200010902BA
:100070004300020100803209040000010202010075
:1000800005240010010424020205240600010524B1
:100090000103010705830308000209040100020AA5
:1000A00000000007050102080000070581020800A2
:1000B000000011241FBECFE5D4E0DEBFCDBF10E0AD
:1000C000A0E6B0E0E4E6FBE002C005900D92AE369B
:1000D000B107D9F712E0AEE6B0E001C01D92AC3333
:1000E000B107E1F782D43DC58BCF85B7836085BF6B
:1000F0008BB780648BBF83EC80938E0080938300EA
:1001000008951F93DC01162F8091630084FF11C0B6
:100110008091830098E8892780938300912F9150E4
:100120009F3F59F0E4E8F0E08D9181939150E0F722
:1001300004C08AE580936300F1CF612F84E890E0EA
:10014000C1D11C5F109363001F9108951F93DC01C0
:10015000162F8091620084FF11C080918E0098E874
:10016000892780938E00912F91509F3F59F0EFE89F
:10017000F0E08D9181939150E0F704C08AE580937F
:100180006200F1CF612F8FE890E09CD11C5F10934B
:1001900062001F9108950F931F93CF93DF93609197
:1001A0009E00161654F5635080919B00CEEAD0E075
:1001B000C81BD10980919A008F3F09F4B2C08D32DB
:1001C00009F475C080916E0087FD0BC0CE01E4D3A9
:1001D0008F3F09F4A9C0882309F097C02FEF30E0C2
:1001E00002C020E030E830936E00209360008091E0
:1001F0009E00181614F410929E008091610084FFF6
:1002000029C0809160008F3F29F1682F893008F064
:1002100072C0861B8093600080916E0080FF73C067
:1002200003EC8F5F80936E0087FD86C0662309F420
:100230006FC089E790E072D3682F7727162F693057
:1002400008F496C08FEF809360009EE100937800E1
:100250009093610080B38C7009F016C180B38C70EC
:1002600009F012C180B38C7009F00EC180B38C709C
:1002700009F00AC180B38C7009F006C180B38C709C
:1002800009F002C180B38C7009F0FEC080B38C709D
:1002900009F0FAC080B38C7009F0F6C080B38C709E
:1002A00009F0F2C010929F0010929900EDC08AE50B
:1002B00080936100683009F094CF8881807609F0DE
:1002C0006EC021E830E0109281008981882309F016
:1002D00075C01092820030939D0020939C0022E014
:1002E00030E88F81882309F07ECF8E81821708F055
:1002F0007ACF282F78CF68E0861B809360008091AA
:100300006E0080FD8DCF0BE48CCF20E030E06BCF12
:1003100060E089E790E0D6D094E08FEF80936000B2
:1003200095CFCE0114D363CF809360008EE180938C
:1003300061002FEF30E057CF20919C0030919D005D
:1003400086FD1FC0462F41504F3F61F0F901942FA9
:10035000A9E7B0E081918D939150E0F7240F311D12
:100360002F5F3F4F30939D0020939C00772766CFEF
:1003700089E790E0A7D0912F9C5F183008F066CFF6
:10038000CCCF462F41504F3F69F3F901942FA9E795
:10039000B0E084918D9331969150D8F7DFCFCE01A4
:1003A0009AD2282F30E82F3F09F09BCF888187FD14
:1003B00002C03F7718CF2E813F7715CF853069F087
:1003C000863089F08830D9F0893011F18A3031F1E6
:1003D0008B3081F120E030E884CF8A8180939F00C8
:1003E00020E030E87ECF8B818130F9F08230E9F077
:1003F000833041F18132C9F020E030EC72CF81EAE4
:1004000090E090939D0080939C0021E030E869CFBC
:100410008A818093A10020E030E863CF30939D0073
:1004200020939C0021E030E85CCFCE013ED2282F03
:1004300030ECB9CF83EC80938E008093830020E072
:1004400030E84FCF8A81882349F486E290E0909388
:100450009D0080939C0024E030EC43CF813059F024
:10046000823051F68CE490E090939D0080939C0044
:1004700020E130EC36CF8AE290E090939D008093AB
:100480009C0022E230EC2DCFDF91CF911F910F9194
:100490000895A82FB92F8FEF9FEF41E050EA6150E8
:1004A00070F02D9138E0722F7827969587952695D4
:1004B00070FF02C0842795273A95A9F7F0CF809561
:1004C00090950895E6DF8D939D930895CF93CFB7D0
:1004D000CF93839BFECF839B09C0839B07C0839BE5
:1004E00005C0839B03C0839B01C09EC0DF93C09166
:1004F0009B00DD27CE55DF4F839B02C0DF91EBCF02
:100500002F930F931F9300B32FEF03FB20F94F930B
:100510003F9310B34FEF012703FB21F93BE031C0BC
:100520004E7F012F10B3216028C0102F4D7F226015
:10053000000000B329C04B7F2460012F000010B3DE
:100540002BC010B3477F28602AC04F7E00B32061C4
:100550002CC04F7D10B320622FC04F7B00B32064AE
:1005600032C0422700B349934FEF0000102713FB1E
:1005700020F910B31C70A9F1297F91F2012703FB28
:1005800021F900B3237F89F23150F0F1102713FBDA
:1005900022F910B3277E79F2012703FB23F92F7C80
:1005A00081F200B3102713FB24F92F7971F200C0F8
:1005B00010B3012703FB25F92F7359F200C000B3D4
:1005C000102713FB26F9223040F200C010B3012798
:1005D00003FB27F9243028F64F77206810B300007A
:1005E000F9CF3B503195333010E41ABFB8F0C31B3C
:1005F000D0400881033C99F10B3489F11981412FD6
:100600001F7720919900121731F40936E9F10D3264
:10061000C1F0013EB1F022272093A0003F914F91FD
:100620001F910F912F91DF91CF91CFBFCF9118954F
:100630003091630034FD56C000936300C3E8D0E0FE
:1006400055C047FD0FEF0093A0003F914F911F91C0
:100650000F912F91DF91CAB7C6FD3BCFE5CF009137
:10066000A0000023D9F210919E001123B9F5343077
:10067000BAF130939E0000939A0010919B003BE0EA
:10068000311B30939B002CC000919E00013034F54B
:100690000AE547FD09C03091610034FD23C0009395
:1006A0006100C8E7D0E022C01A8110FDC1CF3091AF
:1006B000620034FD17C000936200CEE8D0E016C09F
:1006C000052710E002BB1FC0052722C0052727C051
:1006D00005272CC0052710E002BB33C04AE503C044
:1006E00042ED01C0432FC4E1D0E032E011B31C6001
:1006F000939A02B311BB5F935CE020E820FF0527CB
:1007000002BB279517951C3FD8F620FF0527279594
:1007100002BB17951C3FC0F620FF052727951795AC
:1007200002BB1C3F98F620FF0527279517951C3F15
:1007300002BB70F600C0499120FF052702BB279538
:1007400017951C3F38F620FF0527279502BB179504
:100750001C3F38F520FF05272795179502BB1C3F46
:1007600010F520FF0527279517951C3F02BBE8F4DD
:10077000242F3A9519F6037F5F9102BB00C01091B8
:100780009F00C651D04011F01093990010E41ABF99
:10079000086011B3137F402F437F02BB11BB42BBE4
:1007A0003DCF0527D3CF0527D8CF0527DDCFBF9273
:1007B000CF92DF92EF92FF920F931F936B017C0118
:1007C000B42E122FCC0CDD1CEE1CFF1CCC0CDD1C3F
:1007D000EE1CFF1CCC0CDD1CEE1CFF1C60E07BE162
:1007E00087EB90E0A70196019AD12150304040401C
:1007F0005040599A1AB881E0B81629F06B2D6295CD
:10080000607F606801C060EB1695110F110F110F2A
:10081000802F99270597880F991F182B612B60BD92
:1008200029B930BD88E18AB91F910F91FF90EF90EF
:10083000DF90CF90BF9008955D9B15C020913A0244
:1008400090913B02291779F0E92FFF27E754FE4FDB
:1008500080818CB9E92FEF5FEF77E0933B028091C5
:100860009E0087FD15C05F9B08958BB12CB18C71E4
:10087000D9F7E091B8019E2F9F5F809139029817B8
:1008800099F3FF27E854FF4F20839093B801089510
:10089000E21BE150EF77E93030F310929E00E3CF96
:1008A0008BB19927807890700895FC018381813005
:1008B00049F08EE690E090939D0080939C0083E445
:1008C00090E008958CE590E090939D0080939C00CB
:1008D00082E190E00895FC012081822F80768032B1
:1008E000B9F49181892F80528230A8F0923241F080
:1008F00027FD0EC081E080936F0080E090E00895B6
:10090000809170008823A1F782E080937000F0CF7F
:1009100080E090E008958FEF90E00895FC018091D1
:10092000740080838091750081838091760082833A
:10093000809177008383809171008483809172001D
:10094000858380917300868387E090E00895DC01C1
:100950006623E9F090913B02E0913A022D91EF5F1E
:100960008E2F8F77E150891739F0FF27E754FE4F1C
:100970002083E82F80933A02615081F79E1B9150AB
:100980009F77993018F48FEF80939E00089590918F
:100990003B02E0913A02F2CF0F93FC0180818093F9
:1009A00074008181809375008281809376008381B9
:1009B000809377006091740070917500809176004B
:1009C0009091770000917300209171004091720026
:1009D000EEDE10923B021092B80110923902109292
:1009E0003A0281E090E00F9108950F9388E190E042
:1009F0002EE00FB6F894A89581BD0FBE21BD83EF00
:100A000082BB8CE081BB9EEF8FEF9150F1F781505C
:100A1000E1F711BA80EC92E1A0E0B0E080937400BD
:100A200090937500A0937600B093770010927100B8
:100A30001092720088E08093730008E020E040E0AC
:100A400060EC72E180E090E0B2DE10923B02109226
:100A5000B8011092390210923A0247DB8BE480937E
:100A60008E00809383001092700010926F00789433
:100A7000A89591DBE1DE8091620084FF1DC090911A
:100A800039028091B8018917B8F1891B282F3327C3
:100A9000022F2223C1F580916F00882369F0109204
:100AA0006F00892F9927602F88549F4F4FDB8091CB
:100AB0003902080F00933902909170009923C1F216
:100AC0008091630084FFD4CF923021F162E08CE604
:100AD00090E017DB80917000815080937000A895A2
:100AE0005ADBAADE8091620084FFE6CF9091390242
:100AF0008091B801891748F6892F8195282F3327CF
:100B0000022F222341F2283050F281E080936F00BF
:100B100008E0C7CF68E084E690E0F3DADBCFA1E23B
:100B20001A2EAA1BBB1BFD010DC0AA1FBB1FEE1F67
:100B3000FF1FA217B307E407F50720F0A21BB30BB2
:100B4000E40BF50B661F771F881F991F1A9469F72E
:100B500060957095809590959B01AC01BD01CF018A
:040B60000895FFCF26
:0E0B6400FF5A5A5AA1200000000002000300B0
:00000001FF
